:1000000009C021C020C01FC01EC01DC01CC01BC015
:1000100057C119C011241FBECFE9CDBF10E0A0E623
:10002000B0E0E2EEF3E002C005900D92AA36B1070F
:10003000D9F710E0AAE6B0E001C01D92AA37B107D7
:10004000E1F758D0CCC1DCCF90E80FB6F89496BD5C
:1000500086BD0FBE08950895CF92DF92EF92FF9272
:100060000F931F93082F10E0C80141969AD1F82EE4
:10007000C801429696D1E82EC801439692D120E05D
:10008000CC24CA940F2DDD2460EB74E0FF0CFF0C30
:1000900010E0482F50E0A8E7B0E015C0C9BC802FA1
:1000A0009D2D04C0FB013197F1F701970097D1F71F
:1000B00019BC8F2D912F04C0FB013197F1F70197E7
:1000C0000097D1F72F5F2E1548F39A0109C080E100
:1000D00097E2FD013197F1F70197D9F721503040B0
:1000E00021153105A1F720E0EECF90E0419659D1DE
:1000F00089BDFFCFFF920F931F938AE690E060E0E7
:1001000070E04EE050E03ED180917100E82FF0E0C9
:10011000E659FF4F00858F5F833008F080E0E82FBD
:10012000F0E0E659FF4F91E0908780937100809155
:100130006E00882381F480917000863060F0909387
:100140006E008FEF80936F0010926D001092700020
:10015000FF24F39401C0FF2480916E00882311F4E2
:1001600010E01AC0002361F080916F008F5F8093D0
:100170006F008C3010F010926F0010916F000CC067
:1001800010926E0080916F0080936C0081E08093EC
:100190006D0010E0FF24F39480916D00882381F1BD
:1001A000843028F4823050F4813009F505C0843061
:1001B00059F08530E1F40EC082E003C0013041F413
:1001C0008F5F80936D001AC0023011F485E0F9CF83
:1001D00086E0F7CF013059F480916B0060916C009C
:1001E00090E0FC01E659FF4F63870B96EAD010922E
:1001F0006D008FEF80936B0080936C001092700005
:1002000080916E00882311F5002349F080916A00E7
:100210008F5F80936A00809170008F5F09C080912A
:100220006D00882321F480916A0080936B0081E047
:100230008093700080916A00833010F010926A0001
:10024000E0916A00F0E0E659FF4F13858AE690E0FE
:1002500060E070E04BE050E0ACD0B99A81E28FBD35
:1002600081E083BFFF2081F080E69AEEFC013197A8
:10027000F1F729B5209529BDFC013197F1F729B592
:10028000209529BD0197F1F71C3008F010E0110FFF
:10029000110F812F90E0409684D0E82FF894A89514
:1002A00088E181BD84E481BD7894F0E0EE0FFF1F0A
:1002B000E05AFF4F0190F081E02D812F0995FFCF8B
:1002C0001F920F920FB60F9211242F933F934F93CB
:1002D0005F936F937F938F939F93AF93BF93EF93AE
:1002E000FF9320917800283008F03BC08091710086
:1002F00090E008962F5F20937800243041F028305A
:1003000019F0213071F516C060E05BD02AC062E0C0
:1003100058D080916D00843021F589B5805889BD11
:1003200088EE93E028E730E0F9013197F1F7019783
:10033000D9F714C090916D00892F8250823010F04F
:10034000953079F489B5805889BD88EE93E028E727
:1003500030E0F9013197F1F70197D9F789B5805865
:1003600089BDFF91EF91BF91AF919F918F917F9147
:100370006F915F914F913F912F910F900FBE0F9012
:100380001F901895A82F862FE82FE199FECF1FBA4E
:1003900005C0EEBBE09AE3950DB20D924150C8F74F
:1003A0000895E199FECF1FBA8EBBE09A99278DB3CD
:1003B0000895A82F862F02C02D9104D04150E0F758
:1003C0000895262FE199FECF1CBA1FBA8EBB2DBB14
:1003D0000FB6F894E29AE19A0FBE01960895F89448
:0203E000FFCF4D
:0A03E20075002C002B002B002B00EF
:00000001FF
